 objmonusage006

 Timestamp is 6be89054 (reproducible build file hash)

 Preferred load address is 0000000180000000

 Start         Length     Name                   Class
 0001:00000000 000029d0H .text$mn                CODE
 0001:000029d0 00000036H .text$mn$00             CODE
 0001:00002a06 00000092H .text$x                 CODE
 0002:00000000 00000190H .idata$5                DATA
 0002:00000190 00000038H .00cfg                  DATA
 0002:000001c8 00000008H .CRT$XCA                DATA
 0002:000001d0 00000008H .CRT$XCZ                DATA
 0002:000001d8 00000008H .CRT$XIA                DATA
 0002:000001e0 00000008H .CRT$XIC                DATA
 0002:000001e8 00000008H .CRT$XIZ                DATA
 0002:000001f0 00000008H .CRT$XLA                DATA
 0002:000001f8 00000008H .CRT$XLZ                DATA
 0002:00000200 00000008H .CRT$XPA                DATA
 0002:00000208 00000008H .CRT$XPZ                DATA
 0002:00000210 00000008H .CRT$XTA                DATA
 0002:00000218 00000008H .CRT$XTZ                DATA
 0002:00000220 00000000H .gehcont$y              DATA
 0002:00000220 00000000H .gfids$y                DATA
 0002:00000220 00001a60H .rdata                  DATA
 0002:00001c80 00000000H .rdata$CastGuardVftablesA DATA
 0002:00001c80 00000000H .rdata$CastGuardVftablesC DATA
 0002:00001c80 00000028H .rdata$T                DATA
 0002:00001ca8 000000b0H .rdata$voltmd           DATA
 0002:00001d58 00000320H .rdata$zzzdbg           DATA
 0002:00002078 00000008H .rtc$IAA                DATA
 0002:00002080 00000008H .rtc$IZZ                DATA
 0002:00002088 00000008H .rtc$TAA                DATA
 0002:00002090 00000008H .rtc$TZZ                DATA
 0002:00002098 00000004H .tls                    DATA
 0002:0000209c 00000004H .tls$                   DATA
 0002:000020a0 00000008H .tls$ZZZ                DATA
 0002:000020a8 000002d8H .xdata                  DATA
 0002:00002380 000003f0H .edata                  DATA
 0002:00002770 00000064H .idata$2                DATA
 0002:000027d4 00000014H .idata$3                DATA
 0002:000027e8 00000190H .idata$4                DATA
 0002:00002978 00000414H .idata$6                DATA
 0003:00000000 00000080H .data                   DATA
 0003:00000080 0001b248H .bss                    DATA
 0004:00000000 0000036cH .pdata                  DATA

  Address         Publics by Value              Rva+Base               Lib:Object

 0000:00000000       __AbsoluteZero             0000000000000000     <absolute>
 0000:00000000       ___safe_se_handler_count   0000000000000000     <absolute>
 0000:00000000       ___safe_se_handler_table   0000000000000000     <absolute>
 0000:00000000       __arm64x_extra_rfe_table   0000000000000000     <absolute>
 0000:00000000       __arm64x_extra_rfe_table_size 0000000000000000     <absolute>
 0000:00000000       __arm64x_native_entrypoint 0000000000000000     <absolute>
 0000:00000000       __arm64x_redirection_metadata 0000000000000000     <absolute>
 0000:00000000       __arm64x_redirection_metadata_count 0000000000000000     <absolute>
 0000:00000000       __dynamic_value_reloc_table 0000000000000000     <absolute>
 0000:00000000       __enclave_config           0000000000000000     <absolute>
 0000:00000000       __guard_check_icall_a64n_fptr 0000000000000000     <absolute>
 0000:00000000       __guard_eh_cont_count      0000000000000000     <absolute>
 0000:00000000       __guard_eh_cont_table      0000000000000000     <absolute>
 0000:00000000       __guard_fids_count         0000000000000000     <absolute>
 0000:00000000       __guard_fids_table         0000000000000000     <absolute>
 0000:00000000       __guard_iat_count          0000000000000000     <absolute>
 0000:00000000       __guard_iat_table          0000000000000000     <absolute>
 0000:00000000       __guard_longjmp_count      0000000000000000     <absolute>
 0000:00000000       __guard_longjmp_table      0000000000000000     <absolute>
 0000:00000000       __hybrid_auxiliary_iat     0000000000000000     <absolute>
 0000:00000000       __hybrid_auxiliary_iat_copy 0000000000000000     <absolute>
 0000:00000000       __hybrid_code_map          0000000000000000     <absolute>
 0000:00000000       __hybrid_code_map_count    0000000000000000     <absolute>
 0000:00000000       __x64_code_ranges_to_entry_points 0000000000000000     <absolute>
 0000:00000000       __x64_code_ranges_to_entry_points_count 0000000000000000     <absolute>
 0000:00000100       __guard_flags              0000000000000100     <absolute>
 0000:00000000       __ImageBase                0000000180000000     <linker-defined>
 0001:00000000       ?NewObject@JNIEnv_@@QEAAPEAV_jobject@@PEAV_jclass@@PEAU_jmethodID@@ZZ 0000000180001000 f i libobjmonusage006.obj
 0001:00000024       ?TranslateError@@YAPEBDW4jvmtiError@@@Z 0000000180001024 f   libobjmonusage006.obj
 0001:000002dc       ?nsk_jni_check_exception@@YAHPEAUJNIEnv_@@QEBDH@Z 00000001800012dc f   libobjmonusage006.obj
 0001:00000420       ?nsk_jni_lverify@@YAHHPEAUJNIEnv_@@HQEBDH1ZZ 0000000180001420 f   libobjmonusage006.obj
 0001:000004c0       Agent_Initialize           00000001800014c0 f   libobjmonusage006.obj
 0001:000005ac       Agent_OnAttach             00000001800015ac f   libobjmonusage006.obj
 0001:000005ac       Agent_OnLoad               00000001800015ac f   libobjmonusage006.obj
 0001:000005b4       Java_nsk_jvmti_GetObjectMonitorUsage_objmonusage006_check 00000001800015b4 f   libobjmonusage006.obj
 0001:00000610       Java_nsk_jvmti_GetObjectMonitorUsage_objmonusage006_getRes 0000000180001610 f   libobjmonusage006.obj
 0001:00000618       Java_nsk_jvmti_unit_FollowReferences_FollowRefObjects_addRefToVerify 0000000180001618 f   libobjmonusage006.obj
 0001:000007d4       Java_nsk_jvmti_unit_FollowReferences_FollowRefObjects_getTag 00000001800017d4 f   libobjmonusage006.obj
 0001:00000890       Java_nsk_jvmti_unit_FollowReferences_FollowRefObjects_resetRefsToVerify 0000000180001890 f   libobjmonusage006.obj
 0001:00000898       Java_nsk_jvmti_unit_FollowReferences_FollowRefObjects_resetTags 0000000180001898 f   libobjmonusage006.obj
 0001:000008dc       Java_nsk_jvmti_unit_FollowReferences_FollowRefObjects_setTag 00000001800018dc f   libobjmonusage006.obj
 0001:00000b28       Java_nsk_share_jvmti_ArgumentHandler_getAgentOptionsString 0000000180001b28 f   libobjmonusage006.obj
 0001:00000bd4       Java_nsk_share_jvmti_DebugeeClass_checkStatus 0000000180001bd4 f   libobjmonusage006.obj
 0001:00000c5c       Java_nsk_share_jvmti_DebugeeClass_resetAgentData 0000000180001c5c f   libobjmonusage006.obj
 0001:00000cbc       Java_nsk_share_jvmti_RedefineAgent_agentStatus 0000000180001cbc f   libobjmonusage006.obj
 0001:00000cc8       Java_nsk_share_jvmti_RedefineAgent_isRedefined 0000000180001cc8 f   libobjmonusage006.obj
 0001:00000cd4       Java_nsk_share_jvmti_RedefineAgent_redefineAttempted 0000000180001cd4 f   libobjmonusage006.obj
 0001:00000ce0       MA_checkStatus             0000000180001ce0 f   libobjmonusage006.obj
 0001:00000d84       __local_stdio_printf_options 0000000180001d84 f i libobjmonusage006.obj
 0001:00000f54       exitOnError                0000000180001f54 f   libobjmonusage006.obj
 0001:00001008       fprintf                    0000000180002008 f i libobjmonusage006.obj
 0001:0000104c       nsk_jvmti_lverify          000000018000204c f   libobjmonusage006.obj
 0001:0000113c       nsk_jvmti_resetAgentData   000000018000213c f   libobjmonusage006.obj
 0001:000011b0       nsk_lcomplain              00000001800021b0 f   libobjmonusage006.obj
 0001:000011d0       nsk_ldisplay               00000001800021d0 f   libobjmonusage006.obj
 0001:000011f0       nsk_ltrace                 00000001800021f0 f   libobjmonusage006.obj
 0001:00001210       nsk_lvcomplain             0000000180002210 f   libobjmonusage006.obj
 0001:000013c8       nsk_lvdisplay              00000001800023c8 f   libobjmonusage006.obj
 0001:00001414       nsk_lverify                0000000180002414 f   libobjmonusage006.obj
 0001:00001470       nsk_lvtrace                0000000180002470 f   libobjmonusage006.obj
 0001:000014d0       nsk_printf                 00000001800024d0 f   libobjmonusage006.obj
 0001:000014f8       nsk_vprintf                00000001800024f8 f   libobjmonusage006.obj
 0001:000015ac       printf                     00000001800025ac f i libobjmonusage006.obj
 0001:00001aac       __raise_securityfailure    0000000180002aac f   MSVCRT:gs_report.obj
 0001:00001ae0       __report_gsfailure         0000000180002ae0 f   MSVCRT:gs_report.obj
 0001:00001d20       __GSHandlerCheck           0000000180002d20 f   MSVCRT:gshandler.obj
 0001:00001d40       __GSHandlerCheckCommon     0000000180002d40 f   MSVCRT:gshandler.obj
 0001:00001db0       __security_check_cookie    0000000180002db0 f   MSVCRT:amdsecgs.obj
 0001:000020f0       _DllMainCRTStartup         00000001800030f0 f   MSVCRT:dll_dllmain.obj
 0001:00002130       __scrt_acquire_startup_lock 0000000180003130 f   MSVCRT:utility.obj
 0001:0000216c       __scrt_dllmain_after_initialize_c 000000018000316c f   MSVCRT:utility.obj
 0001:000021a0       __scrt_dllmain_before_initialize_c 00000001800031a0 f   MSVCRT:utility.obj
 0001:000021b8       __scrt_dllmain_crt_thread_attach 00000001800031b8 f   MSVCRT:utility.obj
 0001:000021e0       __scrt_dllmain_crt_thread_detach 00000001800031e0 f   MSVCRT:utility.obj
 0001:000021f8       __scrt_dllmain_exception_filter 00000001800031f8 f   MSVCRT:utility.obj
 0001:00002258       __scrt_dllmain_uninitialize_c 0000000180003258 f   MSVCRT:utility.obj
 0001:00002288       __scrt_dllmain_uninitialize_critical 0000000180003288 f   MSVCRT:utility.obj
 0001:0000229c       __scrt_initialize_crt      000000018000329c f   MSVCRT:utility.obj
 0001:000022e8       __scrt_initialize_onexit_tables 00000001800032e8 f   MSVCRT:utility.obj
 0001:00002374       __scrt_is_nonwritable_in_current_image 0000000180003374 f   MSVCRT:utility.obj
 0001:0000240c       __scrt_release_startup_lock 000000018000340c f   MSVCRT:utility.obj
 0001:00002430       __scrt_uninitialize_crt    0000000180003430 f   MSVCRT:utility.obj
 0001:0000245c       _onexit                    000000018000345c f   MSVCRT:utility.obj
 0001:00002498       atexit                     0000000180003498 f   MSVCRT:utility.obj
 0001:000024b0       __crt_debugger_hook        00000001800034b0 f   MSVCRT:utility_desktop.obj
 0001:000024b8       __scrt_fastfail            00000001800034b8 f   MSVCRT:utility_desktop.obj
 0001:00002604       _guard_check_icall_nop     0000000180003604 f i MSVCRT:guard_support.obj
 0001:00002608       __security_init_cookie     0000000180003608 f   MSVCRT:gs_support.obj
 0001:000026b4       DllMain                    00000001800036b4 f   MSVCRT:dll_dllmain_stub.obj
 0001:000026d8       ?__scrt_initialize_type_info@@YAXXZ 00000001800036d8 f   MSVCRT:tncleanup.obj
 0001:000026e8       ?__scrt_uninitialize_type_info@@YAXXZ 00000001800036e8 f   MSVCRT:tncleanup.obj
 0001:000026f4       __local_stdio_scanf_options 00000001800036f4 f i MSVCRT:default_local_stdio_options.obj
 0001:000026fc       __scrt_initialize_default_local_stdio_options 00000001800036fc f   MSVCRT:default_local_stdio_options.obj
 0001:00002718       __scrt_get_dyn_tls_init_callback 0000000180003718 f   MSVCRT:dyn_tls_init.obj
 0001:00002720       _RTC_Initialize            0000000180003720 f   MSVCRT:initsect.obj
 0001:0000275c       _RTC_Terminate             000000018000375c f   MSVCRT:initsect.obj
 0001:00002798       __isa_available_init       0000000180003798 f   MSVCRT:cpu_disp.obj
 0001:00002944       _get_startup_argv_mode     0000000180003944 f   MSVCRT:argv_mode.obj
 0001:0000294c       __scrt_is_ucrt_dll_in_use  000000018000394c f   MSVCRT:ucrt_detection.obj
 0001:00002960       memcpy                     0000000180003960 f   vcruntime:VCRUNTIME140.dll
 0001:00002966       memset                     0000000180003966 f   vcruntime:VCRUNTIME140.dll
 0001:0000296c       strchr                     000000018000396c f   vcruntime:VCRUNTIME140.dll
 0001:00002972       __C_specific_handler       0000000180003972 f   vcruntime:VCRUNTIME140.dll
 0001:00002978       __std_type_info_destroy_list 0000000180003978 f   vcruntime:VCRUNTIME140.dll
 0001:0000297e       strlen                     000000018000397e f   ucrt:api-ms-win-crt-string-l1-1-0.dll
 0001:00002984       _initterm                  0000000180003984 f   ucrt:api-ms-win-crt-runtime-l1-1-0.dll
 0001:0000298a       _initterm_e                000000018000398a f   ucrt:api-ms-win-crt-runtime-l1-1-0.dll
 0001:00002990       _seh_filter_dll            0000000180003990 f   ucrt:api-ms-win-crt-runtime-l1-1-0.dll
 0001:00002996       _configure_narrow_argv     0000000180003996 f   ucrt:api-ms-win-crt-runtime-l1-1-0.dll
 0001:0000299c       _initialize_narrow_environment 000000018000399c f   ucrt:api-ms-win-crt-runtime-l1-1-0.dll
 0001:000029a2       _initialize_onexit_table   00000001800039a2 f   ucrt:api-ms-win-crt-runtime-l1-1-0.dll
 0001:000029a8       _register_onexit_function  00000001800039a8 f   ucrt:api-ms-win-crt-runtime-l1-1-0.dll
 0001:000029ae       _execute_onexit_table      00000001800039ae f   ucrt:api-ms-win-crt-runtime-l1-1-0.dll
 0001:000029b4       _crt_atexit                00000001800039b4 f   ucrt:api-ms-win-crt-runtime-l1-1-0.dll
 0001:000029ba       _cexit                     00000001800039ba f   ucrt:api-ms-win-crt-runtime-l1-1-0.dll
 0001:000029c0       __acrt_initialize          00000001800039c0 f   MSVCRT:ucrt_stubs.obj
 0001:000029c0       __acrt_thread_attach       00000001800039c0 f   MSVCRT:ucrt_stubs.obj
 0001:000029c0       __acrt_thread_detach       00000001800039c0 f   MSVCRT:ucrt_stubs.obj
 0001:000029c0       __acrt_uninitialize        00000001800039c0 f   MSVCRT:ucrt_stubs.obj
 0001:000029c0       __acrt_uninitialize_critical 00000001800039c0 f   MSVCRT:ucrt_stubs.obj
 0001:000029c0       __scrt_stub_for_acrt_initialize 00000001800039c0 f   MSVCRT:ucrt_stubs.obj
 0001:000029c0       __scrt_stub_for_acrt_thread_attach 00000001800039c0 f   MSVCRT:ucrt_stubs.obj
 0001:000029c0       __scrt_stub_for_acrt_thread_detach 00000001800039c0 f   MSVCRT:ucrt_stubs.obj
 0001:000029c0       __scrt_stub_for_acrt_uninitialize 00000001800039c0 f   MSVCRT:ucrt_stubs.obj
 0001:000029c0       __scrt_stub_for_acrt_uninitialize_critical 00000001800039c0 f   MSVCRT:ucrt_stubs.obj
 0001:000029c0       __vcrt_initialize          00000001800039c0 f   MSVCRT:ucrt_stubs.obj
 0001:000029c0       __vcrt_thread_attach       00000001800039c0 f   MSVCRT:ucrt_stubs.obj
 0001:000029c0       __vcrt_thread_detach       00000001800039c0 f   MSVCRT:ucrt_stubs.obj
 0001:000029c0       __vcrt_uninitialize        00000001800039c0 f   MSVCRT:ucrt_stubs.obj
 0001:000029c0       __vcrt_uninitialize_critical 00000001800039c0 f   MSVCRT:ucrt_stubs.obj
 0001:000029c4       __scrt_stub_for_is_c_termination_complete 00000001800039c4 f   MSVCRT:ucrt_stubs.obj
 0001:000029c4       _is_c_termination_complete 00000001800039c4 f   MSVCRT:ucrt_stubs.obj
 0001:000029e0       _guard_dispatch_icall_nop  00000001800039e0 f   MSVCRT:guard_dispatch.obj
 0001:00002a00       _guard_xfg_dispatch_icall_nop 0000000180003a00 f   MSVCRT:guard_xfg_dispatch.obj
 0002:00000000       __imp_RtlCaptureContext    0000000180004000     kernel32:KERNEL32.dll
 0002:00000008       __imp_RtlLookupFunctionEntry 0000000180004008     kernel32:KERNEL32.dll
 0002:00000010       __imp_RtlVirtualUnwind     0000000180004010     kernel32:KERNEL32.dll
 0002:00000018       __imp_UnhandledExceptionFilter 0000000180004018     kernel32:KERNEL32.dll
 0002:00000020       __imp_SetUnhandledExceptionFilter 0000000180004020     kernel32:KERNEL32.dll
 0002:00000028       __imp_GetCurrentProcess    0000000180004028     kernel32:KERNEL32.dll
 0002:00000030       __imp_TerminateProcess     0000000180004030     kernel32:KERNEL32.dll
 0002:00000038       __imp_IsProcessorFeaturePresent 0000000180004038     kernel32:KERNEL32.dll
 0002:00000040       __imp_CloseHandle          0000000180004040     kernel32:KERNEL32.dll
 0002:00000048       __imp_InitializeCriticalSectionAndSpinCount 0000000180004048     kernel32:KERNEL32.dll
 0002:00000050       __imp_DeleteCriticalSection 0000000180004050     kernel32:KERNEL32.dll
 0002:00000058       __imp_CreateEventW         0000000180004058     kernel32:KERNEL32.dll
 0002:00000060       __imp_GetModuleHandleW     0000000180004060     kernel32:KERNEL32.dll
 0002:00000068       __imp_GetProcAddress       0000000180004068     kernel32:KERNEL32.dll
 0002:00000070       __imp_IsDebuggerPresent    0000000180004070     kernel32:KERNEL32.dll
 0002:00000078       __imp_QueryPerformanceCounter 0000000180004078     kernel32:KERNEL32.dll
 0002:00000080       __imp_GetCurrentProcessId  0000000180004080     kernel32:KERNEL32.dll
 0002:00000088       __imp_GetCurrentThreadId   0000000180004088     kernel32:KERNEL32.dll
 0002:00000090       __imp_GetSystemTimeAsFileTime 0000000180004090     kernel32:KERNEL32.dll
 0002:00000098       __imp_DisableThreadLibraryCalls 0000000180004098     kernel32:KERNEL32.dll
 0002:000000a0       __imp_InitializeSListHead  00000001800040a0     kernel32:KERNEL32.dll
 0002:000000a8       \177KERNEL32_NULL_THUNK_DATA 00000001800040a8     kernel32:KERNEL32.dll
 0002:000000b0       __imp_memcpy               00000001800040b0     vcruntime:VCRUNTIME140.dll
 0002:000000b8       __imp_memset               00000001800040b8     vcruntime:VCRUNTIME140.dll
 0002:000000c0       __imp_strchr               00000001800040c0     vcruntime:VCRUNTIME140.dll
 0002:000000c8       __imp___C_specific_handler 00000001800040c8     vcruntime:VCRUNTIME140.dll
 0002:000000d0       __imp___std_type_info_destroy_list 00000001800040d0     vcruntime:VCRUNTIME140.dll
 0002:000000d8       \177VCRUNTIME140_NULL_THUNK_DATA 00000001800040d8     vcruntime:VCRUNTIME140.dll
 0002:000000e0       __imp__errno               00000001800040e0     ucrt:api-ms-win-crt-runtime-l1-1-0.dll
 0002:000000e8       __imp_exit                 00000001800040e8     ucrt:api-ms-win-crt-runtime-l1-1-0.dll
 0002:000000f0       __imp__cexit               00000001800040f0     ucrt:api-ms-win-crt-runtime-l1-1-0.dll
 0002:000000f8       __imp__crt_atexit          00000001800040f8     ucrt:api-ms-win-crt-runtime-l1-1-0.dll
 0002:00000100       __imp__execute_onexit_table 0000000180004100     ucrt:api-ms-win-crt-runtime-l1-1-0.dll
 0002:00000108       __imp__register_onexit_function 0000000180004108     ucrt:api-ms-win-crt-runtime-l1-1-0.dll
 0002:00000110       __imp__initialize_onexit_table 0000000180004110     ucrt:api-ms-win-crt-runtime-l1-1-0.dll
 0002:00000118       __imp__initialize_narrow_environment 0000000180004118     ucrt:api-ms-win-crt-runtime-l1-1-0.dll
 0002:00000120       __imp__configure_narrow_argv 0000000180004120     ucrt:api-ms-win-crt-runtime-l1-1-0.dll
 0002:00000128       __imp__seh_filter_dll      0000000180004128     ucrt:api-ms-win-crt-runtime-l1-1-0.dll
 0002:00000130       __imp__initterm_e          0000000180004130     ucrt:api-ms-win-crt-runtime-l1-1-0.dll
 0002:00000138       __imp__initterm            0000000180004138     ucrt:api-ms-win-crt-runtime-l1-1-0.dll
 0002:00000140       \177api-ms-win-crt-runtime-l1-1-0_NULL_THUNK_DATA 0000000180004140     ucrt:api-ms-win-crt-runtime-l1-1-0.dll
 0002:00000148       __imp___acrt_iob_func      0000000180004148     ucrt:api-ms-win-crt-stdio-l1-1-0.dll
 0002:00000150       __imp_fflush               0000000180004150     ucrt:api-ms-win-crt-stdio-l1-1-0.dll
 0002:00000158       __imp___stdio_common_vsprintf 0000000180004158     ucrt:api-ms-win-crt-stdio-l1-1-0.dll
 0002:00000160       __imp___stdio_common_vfprintf 0000000180004160     ucrt:api-ms-win-crt-stdio-l1-1-0.dll
 0002:00000168       \177api-ms-win-crt-stdio-l1-1-0_NULL_THUNK_DATA 0000000180004168     ucrt:api-ms-win-crt-stdio-l1-1-0.dll
 0002:00000170       __imp__strdup              0000000180004170     ucrt:api-ms-win-crt-string-l1-1-0.dll
 0002:00000170       __imp_strdup               0000000180004170     ucrt:api-ms-win-crt-string-l1-1-0.dll
 0002:00000178       __imp_strlen               0000000180004178     ucrt:api-ms-win-crt-string-l1-1-0.dll
 0002:00000180       __imp_strncpy              0000000180004180     ucrt:api-ms-win-crt-string-l1-1-0.dll
 0002:00000188       \177api-ms-win-crt-string-l1-1-0_NULL_THUNK_DATA 0000000180004188     ucrt:api-ms-win-crt-string-l1-1-0.dll
 0002:00000190       __guard_check_icall_fptr   0000000180004190     MSVCRT:guard_support.obj
 0002:00000198       __guard_xfg_check_icall_fptr 0000000180004198     MSVCRT:guard_support.obj
 0002:000001a0       __guard_dispatch_icall_fptr 00000001800041a0     MSVCRT:guard_support.obj
 0002:000001a8       __guard_xfg_dispatch_icall_fptr 00000001800041a8     MSVCRT:guard_support.obj
 0002:000001b0       __guard_xfg_table_dispatch_icall_fptr 00000001800041b0     MSVCRT:guard_support.obj
 0002:000001b8       __castguard_check_failure_os_handled_fptr 00000001800041b8     MSVCRT:guard_support.obj
 0002:000001c0       __guard_memcpy_fptr        00000001800041c0     vcruntime:softmemtag.obj
 0002:000001c8       __xc_a                     00000001800041c8     MSVCRT:initializers.obj
 0002:000001d0       __xc_z                     00000001800041d0     MSVCRT:initializers.obj
 0002:000001d8       __xi_a                     00000001800041d8     MSVCRT:initializers.obj
 0002:000001e8       __xi_z                     00000001800041e8     MSVCRT:initializers.obj
 0002:000001f0       __xl_a                     00000001800041f0     MSVCRT:tlssup.obj
 0002:000001f8       __xl_z                     00000001800041f8     MSVCRT:tlssup.obj
 0002:00000200       __xp_a                     0000000180004200     MSVCRT:initializers.obj
 0002:00000208       __xp_z                     0000000180004208     MSVCRT:initializers.obj
 0002:00000210       __xt_a                     0000000180004210     MSVCRT:initializers.obj
 0002:00000218       __xt_z                     0000000180004218     MSVCRT:initializers.obj
 0002:00000220       g_refKindStr               0000000180004220     libobjmonusage006.obj
 0002:000003d0       ??_C@_09BPLDFGCI@unknown_0@ 00000001800043d0     libobjmonusage006.obj
 0002:000003e0       ??_C@_0BL@FPNMECJD@JVMTI_HEAP_REFERENCE_CLASS@ 00000001800043e0     libobjmonusage006.obj
 0002:00000400       ??_C@_0BL@FKGKKLNM@JVMTI_HEAP_REFERENCE_FIELD@ 0000000180004400     libobjmonusage006.obj
 0002:00000420       ??_C@_0CD@CAEHCFJF@JVMTI_HEAP_REFERENCE_ARRAY_ELEM@ 0000000180004420     libobjmonusage006.obj
 0002:00000448       ??_C@_0CC@DNEBMCNK@JVMTI_HEAP_REFERENCE_CLASS_LOAD@ 0000000180004448     libobjmonusage006.obj
 0002:00000470       ??_C@_0BN@CJMIPEBB@JVMTI_HEAP_REFERENCE_SIGNERS@ 0000000180004470     libobjmonusage006.obj
 0002:00000490       ??_C@_0CH@HBOIDPEB@JVMTI_HEAP_REFERENCE_PROTECTION@ 0000000180004490     libobjmonusage006.obj
 0002:000004b8       ??_C@_0BP@MDKGDGKL@JVMTI_HEAP_REFERENCE_INTERFACE@ 00000001800044b8     libobjmonusage006.obj
 0002:000004d8       ??_C@_0CC@JJMIHNJH@JVMTI_HEAP_REFERENCE_STATIC_FIE@ 00000001800044d8     libobjmonusage006.obj
 0002:00000500       ??_C@_0CD@IDHEEGID@JVMTI_HEAP_REFERENCE_CONSTANT_P@ 0000000180004500     libobjmonusage006.obj
 0002:00000528       ??_C@_0CA@EFFCHNG@JVMTI_HEAP_REFERENCE_SUPERCLASS@ 0000000180004528     libobjmonusage006.obj
 0002:00000548       ??_C@_0L@PCDFHGCJ@unknown_11@ 0000000180004548     libobjmonusage006.obj
 0002:00000558       ??_C@_0L@NJBICFOK@unknown_12@ 0000000180004558     libobjmonusage006.obj
 0002:00000568       ??_C@_0L@MAADBEKL@unknown_13@ 0000000180004568     libobjmonusage006.obj
 0002:00000578       ??_C@_0L@IPECICGM@unknown_14@ 0000000180004578     libobjmonusage006.obj
 0002:00000588       ??_C@_0L@JGFJLDCN@unknown_15@ 0000000180004588     libobjmonusage006.obj
 0002:00000598       ??_C@_0L@LNHEOAOO@unknown_16@ 0000000180004598     libobjmonusage006.obj
 0002:000005a8       ??_C@_0L@KEGPNBKP@unknown_17@ 00000001800045a8     libobjmonusage006.obj
 0002:000005b8       ??_C@_0L@CDPHMNGA@unknown_18@ 00000001800045b8     libobjmonusage006.obj
 0002:000005c8       ??_C@_0L@DKOMPMCB@unknown_19@ 00000001800045c8     libobjmonusage006.obj
 0002:000005d8       ??_C@_0L@OJGIPJDB@unknown_20@ 00000001800045d8     libobjmonusage006.obj
 0002:000005e8       ??_C@_0CA@KAOFNDEM@JVMTI_HEAP_REFERENCE_JNI_GLOBAL@ 00000001800045e8     libobjmonusage006.obj
 0002:00000608       ??_C@_0CC@HPFAJBK@JVMTI_HEAP_REFERENCE_SYSTEM_CLA@ 0000000180004608     libobjmonusage006.obj
 0002:00000630       ??_C@_0BN@FDEGFOHC@JVMTI_HEAP_REFERENCE_MONITOR@ 0000000180004630     libobjmonusage006.obj
 0002:00000650       ??_C@_0CB@HKIBCMAJ@JVMTI_HEAP_REFERENCE_STACK_LOCA@ 0000000180004650     libobjmonusage006.obj
 0002:00000678       ??_C@_0BP@EAACMMOE@JVMTI_HEAP_REFERENCE_JNI_LOCAL@ 0000000180004678     libobjmonusage006.obj
 0002:00000698       ??_C@_0BM@IJDEOGOE@JVMTI_HEAP_REFERENCE_THREAD@ 0000000180004698     libobjmonusage006.obj
 0002:000006b8       ??_C@_0BL@EDGPPKC@JVMTI_HEAP_REFERENCE_OTHER@ 00000001800046b8     libobjmonusage006.obj
 0002:000006d4       ??_C@_04BCJPDBDA@Code@     00000001800046d4     libobjmonusage006.obj
 0002:000006e0       ??_C@_0BA@OCLMCFKC@LineNumberTable@ 00000001800046e0     libobjmonusage006.obj
 0002:000006f0       ??_C@_0BD@CPAEPILC@LocalVariableTable@ 00000001800046f0     libobjmonusage006.obj
 0002:00000708       ??_C@_0BH@NMBDNHBD@LocalVariableTypeTable@ 0000000180004708     libobjmonusage006.obj
 0002:00000720       ??_C@_0O@HIHEEDNJ@StackMapTable@ 0000000180004720     libobjmonusage006.obj
 0002:00000730       ??_C@_0L@HCDIAMJG@?9?5?$CFs?0?5?$CFd?3?5@ 0000000180004730     libobjmonusage006.obj
 0002:00000740       ??_C@_0JI@HLPECLFI@?$CD?5?4?4?4?6?$CD?5ERROR?3?5too?5many?5complai@ 0000000180004740     libobjmonusage006.obj
 0002:000007e0       ??_C@_0ED@JNEKCCOB@The?5following?5fake?5exception?5st@ 00000001800047e0     libobjmonusage006.obj
 0002:00000828       ??_C@_0CN@FCNMDFBH@nsk?4share?4Fake_Exception_for_RU@ 0000000180004828     libobjmonusage006.obj
 0002:00000858       ??_C@_08PGFFNAEI@?$CI?$CFs?3?$CFd?$CJ?5@ 0000000180004858     libobjmonusage006.obj
 0002:00000868       ??_C@_0DP@IENMAEGI@s?2test?2hotspot?2jtreg?2vmTestbase@ 0000000180004868     libobjmonusage006.obj
 0002:000008a8       ??_C@_0BL@NDJLFFJB@?7at?5nsk_lvcomplain?$CI?$CFs?3?$CFd?$CJ?6@ 00000001800048a8     libobjmonusage006.obj
 0002:000008c8       ??_C@_0BC@JOOKAFKF@?$CD?5ERROR?3?5?$CFs?0?5?$CFd?3?5@ 00000001800048c8     libobjmonusage006.obj
 0002:000008e0       ??_C@_09KJEAHMEH@?$CD?5ERROR?3?5@ 00000001800048e0     libobjmonusage006.obj
 0002:000008ec       ??_C@_02GPIOPFAK@?$DO?$DO@ 00000001800048ec     libobjmonusage006.obj
 0002:000008f0       ??_C@_02FODMEDOG@?$DM?$DM@ 00000001800048f0     libobjmonusage006.obj
 0002:000008f4       ??_C@_02DJGKEECL@?4?4@     00000001800048f4     libobjmonusage006.obj
 0002:000008f8       ??_C@_0O@CJPGJOAF@?9?5?$CFs?0?5?$CFd?3?5?$CFs?5@ 00000001800048f8     libobjmonusage006.obj
 0002:00000908       ??_C@_0CB@IAKPDOIC@?$CD?5?5?5verified?5assertion?5is?5FALSE@ 0000000180004908     libobjmonusage006.obj
 0002:00000930       ??_C@_0CO@LGONDEPD@stdout?3?5fflush?5failed?5?9?5err?$DN?$CFd?5@ 0000000180004930     libobjmonusage006.obj
 0002:00000960       ??_C@_0CO@KBGKJPBD@stderr?3?5fflush?5failed?5?9?5err?$DN?$CFd?5@ 0000000180004960     libobjmonusage006.obj
 0002:00000990       ??_C@_0BB@JCNMKLLK@JVMTI_ERROR_NONE@ 0000000180004990     libobjmonusage006.obj
 0002:000009a8       ??_C@_0BL@LDIMKLPH@JVMTI_ERROR_INVALID_THREAD@ 00000001800049a8     libobjmonusage006.obj
 0002:000009c8       ??_C@_0CB@PJFPAIKJ@JVMTI_ERROR_INVALID_THREAD_GROU@ 00000001800049c8     libobjmonusage006.obj
 0002:000009f0       ??_C@_0BN@LLMKHMNF@JVMTI_ERROR_INVALID_PRIORITY@ 00000001800049f0     libobjmonusage006.obj
 0002:00000a10       ??_C@_0CB@MBOFKAGB@JVMTI_ERROR_THREAD_NOT_SUSPENDE@ 0000000180004a10     libobjmonusage006.obj
 0002:00000a38       ??_C@_0BN@FABOLPBI@JVMTI_ERROR_THREAD_SUSPENDED@ 0000000180004a38     libobjmonusage006.obj
 0002:00000a58       ??_C@_0BN@FDGNOBJM@JVMTI_ERROR_THREAD_NOT_ALIVE@ 0000000180004a58     libobjmonusage006.obj
 0002:00000a78       ??_C@_0BL@GOBIFKNJ@JVMTI_ERROR_INVALID_OBJECT@ 0000000180004a78     libobjmonusage006.obj
 0002:00000a98       ??_C@_0BK@FCMAJPPC@JVMTI_ERROR_INVALID_CLASS@ 0000000180004a98     libobjmonusage006.obj
 0002:00000ab8       ??_C@_0BP@IKLLBKEB@JVMTI_ERROR_CLASS_NOT_PREPARED@ 0000000180004ab8     libobjmonusage006.obj
 0002:00000ad8       ??_C@_0BN@KLPPLKG@JVMTI_ERROR_INVALID_METHODID@ 0000000180004ad8     libobjmonusage006.obj
 0002:00000af8       ??_C@_0BN@BCEKOKND@JVMTI_ERROR_INVALID_LOCATION@ 0000000180004af8     libobjmonusage006.obj
 0002:00000b18       ??_C@_0BM@DFDGPME@JVMTI_ERROR_INVALID_FIELDID@ 0000000180004b18     libobjmonusage006.obj
 0002:00000b38       ??_C@_0BL@NELIEPEC@JVMTI_ERROR_NO_MORE_FRAMES@ 0000000180004b38     libobjmonusage006.obj
 0002:00000b58       ??_C@_0BJ@BDBECFDM@JVMTI_ERROR_OPAQUE_FRAME@ 0000000180004b58     libobjmonusage006.obj
 0002:00000b78       ??_C@_0BK@MIIFNLOB@JVMTI_ERROR_TYPE_MISMATCH@ 0000000180004b78     libobjmonusage006.obj
 0002:00000b98       ??_C@_0BJ@HPCAOILC@JVMTI_ERROR_INVALID_SLOT@ 0000000180004b98     libobjmonusage006.obj
 0002:00000bb8       ??_C@_0BG@CHILOPNI@JVMTI_ERROR_DUPLICATE@ 0000000180004bb8     libobjmonusage006.obj
 0002:00000bd0       ??_C@_0BG@DIEMLHKM@JVMTI_ERROR_NOT_FOUND@ 0000000180004bd0     libobjmonusage006.obj
 0002:00000be8       ??_C@_0BM@NHMCKHOB@JVMTI_ERROR_INVALID_MONITOR@ 0000000180004be8     libobjmonusage006.obj
 0002:00000c08       ??_C@_0BO@PPEDAJGL@JVMTI_ERROR_NOT_MONITOR_OWNER@ 0000000180004c08     libobjmonusage006.obj
 0002:00000c28       ??_C@_0BG@FCAIPEID@JVMTI_ERROR_INTERRUPT@ 0000000180004c28     libobjmonusage006.obj
 0002:00000c40       ??_C@_0CB@EGDBNKOI@JVMTI_ERROR_INVALID_CLASS_FORMA@ 0000000180004c40     libobjmonusage006.obj
 0002:00000c68       ??_C@_0CG@DGKOGIAL@JVMTI_ERROR_CIRCULAR_CLASS_DEFI@ 0000000180004c68     libobjmonusage006.obj
 0002:00000c90       ??_C@_0BP@ICEALPKC@JVMTI_ERROR_FAILS_VERIFICATION@ 0000000180004c90     libobjmonusage006.obj
 0002:00000cb0       ??_C@_0DC@JDACLMIO@JVMTI_ERROR_UNSUPPORTED_REDEFIN@ 0000000180004cb0     libobjmonusage006.obj
 0002:00000ce8       ??_C@_0DE@GKDKNOMJ@JVMTI_ERROR_UNSUPPORTED_REDEFIN@ 0000000180004ce8     libobjmonusage006.obj
 0002:00000d20       ??_C@_0BO@LAFKIOG@JVMTI_ERROR_INVALID_TYPESTATE@ 0000000180004d20     libobjmonusage006.obj
 0002:00000d40       ??_C@_0DH@INDGCLLB@JVMTI_ERROR_UNSUPPORTED_REDEFIN@ 0000000180004d40     libobjmonusage006.obj
 0002:00000d78       ??_C@_0DE@NHEOMMGI@JVMTI_ERROR_UNSUPPORTED_REDEFIN@ 0000000180004d78     libobjmonusage006.obj
 0002:00000db0       ??_C@_0CA@EKPNJOEP@JVMTI_ERROR_UNSUPPORTED_VERSION@ 0000000180004db0     libobjmonusage006.obj
 0002:00000dd0       ??_C@_0BN@OFFMAHHL@JVMTI_ERROR_NAMES_DONT_MATCH@ 0000000180004dd0     libobjmonusage006.obj
 0002:00000df0       ??_C@_0DN@HHBBLAKE@JVMTI_ERROR_UNSUPPORTED_REDEFIN@ 0000000180004df0     libobjmonusage006.obj
 0002:00000e30       ??_C@_0DO@HMBGBGNA@JVMTI_ERROR_UNSUPPORTED_REDEFIN@ 0000000180004e30     libobjmonusage006.obj
 0002:00000e70       ??_C@_0BP@PBECGKHJ@JVMTI_ERROR_UNMODIFIABLE_CLASS@ 0000000180004e70     libobjmonusage006.obj
 0002:00000e90       ??_C@_0BK@CANILEHF@JVMTI_ERROR_NOT_AVAILABLE@ 0000000180004e90     libobjmonusage006.obj
 0002:00000eb0       ??_C@_0CE@INJKMEFK@JVMTI_ERROR_MUST_POSSESS_CAPABI@ 0000000180004eb0     libobjmonusage006.obj
 0002:00000ed8       ??_C@_0BJ@LBFPFPDM@JVMTI_ERROR_NULL_POINTER@ 0000000180004ed8     libobjmonusage006.obj
 0002:00000ef8       ??_C@_0BP@CHJPNNEM@JVMTI_ERROR_ABSENT_INFORMATION@ 0000000180004ef8     libobjmonusage006.obj
 0002:00000f18       ??_C@_0BP@OMFMNLC@JVMTI_ERROR_INVALID_EVENT_TYPE@ 0000000180004f18     libobjmonusage006.obj
 0002:00000f38       ??_C@_0BN@BIBNPHHO@JVMTI_ERROR_ILLEGAL_ARGUMENT@ 0000000180004f38     libobjmonusage006.obj
 0002:00000f58       ??_C@_0BK@KKNDHDCE@JVMTI_ERROR_NATIVE_METHOD@ 0000000180004f58     libobjmonusage006.obj
 0002:00000f78       ??_C@_0BK@PMKCFHAE@JVMTI_ERROR_OUT_OF_MEMORY@ 0000000180004f78     libobjmonusage006.obj
 0002:00000f98       ??_C@_0BK@NNJBDMNB@JVMTI_ERROR_ACCESS_DENIED@ 0000000180004f98     libobjmonusage006.obj
 0002:00000fb8       ??_C@_0BI@GHECLMNC@JVMTI_ERROR_WRONG_PHASE@ 0000000180004fb8     libobjmonusage006.obj
 0002:00000fd0       ??_C@_0BF@OLIHJOII@JVMTI_ERROR_INTERNAL@ 0000000180004fd0     libobjmonusage006.obj
 0002:00000fe8       ??_C@_0BO@EOHGKJHI@JVMTI_ERROR_UNATTACHED_THREAD@ 0000000180004fe8     libobjmonusage006.obj
 0002:00001008       ??_C@_0CA@LKHFDACL@JVMTI_ERROR_INVALID_ENVIRONMENT@ 0000000180005008     libobjmonusage006.obj
 0002:00001028       ??_C@_0BA@MMFHLOKK@?$DMunknown?5error?$DO@ 0000000180005028     libobjmonusage006.obj
 0002:00001038       ??_C@_0CF@CBHOKDB@throwable?5?$DN?5jni?9?$DOExceptionOccur@ 0000000180005038     libobjmonusage006.obj
 0002:00001060       ??_C@_03OFAPEBGM@?$CFs?6@  0000000180005060     libobjmonusage006.obj
 0002:00001068       ??_C@_0DM@LPIGEGNJ@s?2test?2hotspot?2jtreg?2vmTestbase@ 0000000180005068     libobjmonusage006.obj
 0002:000010a8       ??_C@_0CC@NFCNPEPK@Exception?5in?5JNI?5call?5?$CIcleared?$CJ@ 00000001800050a8     libobjmonusage006.obj
 0002:000010d0       ??_C@_0BJ@IBAKFIKF@jni?9?$DOExceptionDescribe?$CI?$CJ@ 00000001800050d0     libobjmonusage006.obj
 0002:000010f0       ??_C@_0BG@GGKALKMH@jni?9?$DOExceptionClear?$CI?$CJ@ 00000001800050f0     libobjmonusage006.obj
 0002:00001108       ??_C@_0CF@JMGFGJLJ@?$CD?5?5?5verified?5JNI?5assertion?5is?5F@ 0000000180005108     libobjmonusage006.obj
 0002:00001130       ??_C@_0CB@MLNJNCLJ@?5?5jvmti?5error?3?5code?$DN?$CFd?0?5name?$DN?$CFs@ 0000000180005130     libobjmonusage006.obj
 0002:00001158       ??_C@_0CD@OHBGDKMK@?$CD?5?5?5jvmti?5error?3?5code?$DN?$CFd?0?5name?$DN@ 0000000180005158     libobjmonusage006.obj
 0002:00001180       ??_C@_0CG@JNNCGPHB@?$CD?5?5?5error?5expected?3?5code?$DN?$CFd?0?5na@ 0000000180005180     libobjmonusage006.obj
 0002:000011b0       ??_C@_0EB@IMGKPCGE@?$CIstr_obj?5?$DN?5jni?9?$DONewStringUTF?$CIco@ 00000001800051b0     libobjmonusage006.obj
 0002:00001200       ??_C@_0EA@HFOGGBCC@s?2test?2hotspot?2jtreg?2vmTestbase@ 0000000180005200     libobjmonusage006.obj
 0002:00001240       ??_C@_05KKCIMGE@error@     0000000180005240     libobjmonusage006.obj
 0002:00001250       ??_C@_0EA@PNBCDMOA@s?2test?2hotspot?2jtreg?2vmTestbase@ 0000000180005250     libobjmonusage006.obj
 0002:00001290       ??_C@_0DI@ILAHDLMP@?$CI?$CKagentThreadProc?$CJ?$CIjvmti_env?0?5a@ 0000000180005290     libobjmonusage006.obj
 0002:000012c8       ??_C@_0BD@KDBALNLB@JVMTI?5agent?5thread@ 00000001800052c8     libobjmonusage006.obj
 0002:000012e0       ??_C@_0BB@NOKBFPFO@java?1lang?1Thread@ 00000001800052e0     libobjmonusage006.obj
 0002:000012f4       ??_C@_06FALKBLGB@?$DMinit?$DO@ 00000001800052f4     libobjmonusage006.obj
 0002:00001300       ??_C@_0BG@IKDDPPGD@?$CILjava?1lang?1String?$DL?$CJV@ 0000000180005300     libobjmonusage006.obj
 0002:00001320       ??_C@_0EB@IFJBFEKC@?$CIthreadClass?5?$DN?5jni_env?9?$DOFindCla@ 0000000180005320     libobjmonusage006.obj
 0002:00001370       ??_C@_0GF@FGFIBKKL@?$CIthreadCtor?5?$DN?5jni_env?9?$DOGetMetho@ 0000000180005370     libobjmonusage006.obj
 0002:000013d8       ??_C@_0DN@NCPDJLOG@?$CIthreadName?5?$DN?5jni_env?9?$DONewStrin@ 00000001800053d8     libobjmonusage006.obj
 0002:00001420       ??_C@_0FE@PFKODBGC@?$CIthreadObject?5?$DN?5jni_env?9?$DONewObj@ 0000000180005420     libobjmonusage006.obj
 0002:00001480       ??_C@_0ED@HOBAHHJI@?$CIthreadGlobalRef?5?$DN?5jni_env?9?$DONew@ 0000000180005480     libobjmonusage006.obj
 0002:000014d0       ??_C@_0FN@HNJJAHFC@jvmti_env?9?$DORunAgentThread?$CIagent@ 00000001800054d0     libobjmonusage006.obj
 0002:00001530       ??_C@_0EA@MOJDNKDF@Debuggee?5status?5sync?5aborted?5be@ 0000000180005530     libobjmonusage006.obj
 0002:00001570       ??_C@_0EA@EEOEJAEN@status?5?$DN?5syncDebuggeeStatus?$CIjni@ 0000000180005570     libobjmonusage006.obj
 0002:000015b0       ??_C@_0BL@JBCFNBMB@nsk_jvmti_resetAgentData?$CI?$CJ@ 00000001800055b0     libobjmonusage006.obj
 0002:000015d0       ??_C@_0EL@LPBEELIP@s?2test?2hotspot?2jtreg?2vmTestbase@ 00000001800055d0     libobjmonusage006.obj
 0002:00001620       ??_C@_0CK@JDAMFDMJ@jvmti?9?$DOSetTag?$CIo?0?5tag?$CJ?5?$DN?$DN?5JVMTI_@ 0000000180005620     libobjmonusage006.obj
 0002:00001650       ??_C@_0CC@DAMNHKNI@Can?8t?5set?5tag?5?$CFli?5for?5object?5?$CFl@ 0000000180005650     libobjmonusage006.obj
 0002:00001678       ??_C@_0DL@HAJPNKEF@jvmti?9?$DOGetObjectHashCode?$CIo?0?5?$CGha@ 0000000180005678     libobjmonusage006.obj
 0002:000016b8       ??_C@_0BL@JFPIEOBF@Can?8t?5get?5hash?5object?5?$CFlx?6@ 00000001800056b8     libobjmonusage006.obj
 0002:000016d8       ??_C@_0BG@DICPHBKN@setTag?3?5?$CF08x?5?$DM?9?5?$CF?53li@ 00000001800056d8     libobjmonusage006.obj
 0002:000016f0       ??_C@_0DH@FCEEBDMJ@?$CIs?5?$DN?5jni?9?$DOGetStringUTFChars?$CIsIn@ 00000001800056f0     libobjmonusage006.obj
 0002:00001728       ??_C@_0BJ@OKKGHDCN@Can?8t?5get?5string?5at?5?$CF?$CDp?6@ 0000000180005728     libobjmonusage006.obj
 0002:00001748       ??_C@_0BP@EKFLGGFJ@Can?8t?5get?5string?5at?5?$CF?$CDp?3?5null?6@ 0000000180005748     libobjmonusage006.obj
 0002:00001768       ??_C@_06ICODBHCL@?5?1?1?5?$CFs@ 0000000180005768     libobjmonusage006.obj
 0002:00001770       ??_C@_0DB@KGFPLEGO@?$CIr?5?$DN?5jvmti?9?$DOGetTag?$CIo?0?5?$CGtag?$CJ?$CJ?5?$DN?$DN@ 0000000180005770     libobjmonusage006.obj
 0002:000017a8       ??_C@_0CO@PDAGBCGJ@Can?8t?5GetTag?5for?5object?5?$CFlx?4?5Re@ 00000001800057a8     libobjmonusage006.obj
 0002:000017d8       ??_C@_0CH@HPEODOHC@TEST_BUG?3?5Max?4?5number?5of?5refs?5r@ 00000001800057d8     libobjmonusage006.obj
 0002:00001800       ??_C@_0DI@PHFCABIM@?$CIr?5?$DN?5jvmti?9?$DOGetTag?$CIfrom?0?5?$CGtagFr@ 0000000180005800     libobjmonusage006.obj
 0002:00001838       ??_C@_0DI@MDEGFNKD@TEST_BUG?3?5Can?8t?5GetTag?5for?5obje@ 0000000180005838     libobjmonusage006.obj
 0002:00001870       ??_C@_0DE@MLELJAHM@?$CIr?5?$DN?5jvmti?9?$DOGetTag?$CIto?0?5?$CGtagTo?$CJ?$CJ@ 0000000180005870     libobjmonusage006.obj
 0002:000018a8       ??_C@_0CK@DEFLIKCM@Wrong?5result?5of?5a?5valid?5call?5to@ 00000001800058a8     libobjmonusage006.obj
 0002:000018d8       ??_C@_0DG@LAJPGIIE@?$CIGetPotentialCapabilities?$CJ?5unex@ 00000001800058d8     libobjmonusage006.obj
 0002:00001910       ??_C@_0CN@LKPEOJPO@?$CIAddCapabilities?$CJ?5unexpected?5er@ 0000000180005910     libobjmonusage006.obj
 0002:00001940       ??_C@_0CN@BCCBOHCH@?$CIGetCapabilities?$CJ?5unexpected?5er@ 0000000180005940     libobjmonusage006.obj
 0002:00001970       ??_C@_0DD@NPGKGIKA@Warning?3?5GetObjectMonitorUsage?5@ 0000000180005970     libobjmonusage006.obj
 0002:000019a8       ??_C@_0DD@CJKKNKKC@?$CIGetObjectMonitorUsage?$CJ?5unexpec@ 00000001800059a8     libobjmonusage006.obj
 0002:000019f0       ??_C@_1EC@JIJBPKFM@?$AAa?$AAp?$AAi?$AA?9?$AAm?$AAs?$AA?9?$AAw?$AAi?$AAn?$AA?9?$AAc?$AAo?$AAr?$AAe@ 00000001800059f0     MSVCRT:thread_safe_statics.obj
 0002:00001a38       ??_C@_1BK@MGMFAEKH@?$AAk?$AAe?$AAr?$AAn?$AAe?$AAl?$AA3?$AA2?$AA?4?$AAd?$AAl?$AAl@ 0000000180005a38     MSVCRT:thread_safe_statics.obj
 0002:00001a58       ??_C@_0BJ@JEBJOJFJ@SleepConditionVariableCS@ 0000000180005a58     MSVCRT:thread_safe_statics.obj
 0002:00001a78       ??_C@_0BJ@PGPPEPCC@WakeAllConditionVariable@ 0000000180005a78     MSVCRT:thread_safe_statics.obj
 0002:00001a98       _pDefaultRawDllMain        0000000180005a98     MSVCRT:dll_dllmain.obj
 0002:00001a98       _pRawDllMain               0000000180005a98     MSVCRT:dll_dllmain.obj
 0002:00001aa0       __xmm@ffffffffffffffffffffffffffffffff 0000000180005aa0     MSVCRT:utility.obj
 0002:00001ab0       _load_config_used          0000000180005ab0     MSVCRT:loadcfg.obj
 0002:00001c80       _tls_used                  0000000180005c80     MSVCRT:tlssup.obj
 0002:00001ca8       __volatile_metadata        0000000180005ca8     <linker-defined>
 0002:00002078       __rtc_iaa                  0000000180006078     MSVCRT:initsect.obj
 0002:00002080       __rtc_izz                  0000000180006080     MSVCRT:initsect.obj
 0002:00002088       __rtc_taa                  0000000180006088     MSVCRT:initsect.obj
 0002:00002090       __rtc_tzz                  0000000180006090     MSVCRT:initsect.obj
 0002:00002098       _tls_start                 0000000180006098     MSVCRT:tlssup.obj
 0002:0000209c       _Init_thread_epoch         000000018000609c     MSVCRT:thread_safe_statics.obj
 0002:000020a0       _tls_end                   00000001800060a0     MSVCRT:tlssup.obj
 0002:00002770       __IMPORT_DESCRIPTOR_KERNEL32 0000000180006770     kernel32:KERNEL32.dll
 0002:00002784       __IMPORT_DESCRIPTOR_VCRUNTIME140 0000000180006784     vcruntime:VCRUNTIME140.dll
 0002:00002798       __IMPORT_DESCRIPTOR_api-ms-win-crt-runtime-l1-1-0 0000000180006798     ucrt:api-ms-win-crt-runtime-l1-1-0.dll
 0002:000027ac       __IMPORT_DESCRIPTOR_api-ms-win-crt-stdio-l1-1-0 00000001800067ac     ucrt:api-ms-win-crt-stdio-l1-1-0.dll
 0002:000027c0       __IMPORT_DESCRIPTOR_api-ms-win-crt-string-l1-1-0 00000001800067c0     ucrt:api-ms-win-crt-string-l1-1-0.dll
 0002:000027d4       __NULL_IMPORT_DESCRIPTOR   00000001800067d4     kernel32:KERNEL32.dll
 0003:00000030       _Init_global_epoch         0000000180007030     MSVCRT:thread_safe_statics.obj
 0003:00000040       __security_cookie          0000000180007040     MSVCRT:gs_cookie.obj
 0003:00000048       __security_cookie_complement 0000000180007048     MSVCRT:gs_cookie.obj
 0003:00000050       __scrt_native_dllmain_reason 0000000180007050     MSVCRT:utility.obj
 0003:00000058       __isa_available            0000000180007058     MSVCRT:cpu_disp.obj
 0003:0000005c       __isa_enabled              000000018000705c     MSVCRT:cpu_disp.obj
 0003:00000060       __memset_fast_string_threshold 0000000180007060     MSVCRT:cpu_disp.obj
 0003:00000068       __memset_nt_threshold      0000000180007068     MSVCRT:cpu_disp.obj
 0003:00000070       __scrt_ucrt_dll_is_in_use  0000000180007070     MSVCRT:ucrt_stubs.obj
 0003:00000080       g_wrongHeapCallbacks       0000000180007080     libobjmonusage006.obj
 0003:00000100       g_szTagInfo                0000000180007100     libobjmonusage006.obj
 0003:00002040       g_tagFlags                 0000000180009040     libobjmonusage006.obj
 0003:00002428       g_refsToVerifyCnt          0000000180009428     libobjmonusage006.obj
 0003:0000242c       g_fakeUserData             000000018000942c     libobjmonusage006.obj
 0003:00002430       g_tagVisitCount            0000000180009430     libobjmonusage006.obj
 0003:000033d0       g_refsToVerify             000000018000a3d0     libobjmonusage006.obj
 0003:0001aad0       g_userDataError            0000000180021ad0     libobjmonusage006.obj
 0003:0001ac80       ?_OptionsStorage@?1??__local_stdio_printf_options@@9@4_KA 0000000180021c80     libobjmonusage006.obj
 0003:0001b248       _tls_index                 0000000180022248     MSVCRT:tlssup.obj
 0003:0001b250       __scrt_current_native_startup_state 0000000180022250     MSVCRT:utility.obj
 0003:0001b258       __scrt_native_startup_lock 0000000180022258     MSVCRT:utility.obj
 0003:0001b298       __scrt_debugger_hook_flag  0000000180022298     MSVCRT:utility_desktop.obj
 0003:0001b2a0       ?__type_info_root_node@@3U__type_info_node@@A 00000001800222a0     MSVCRT:tncleanup.obj
 0003:0001b2b0       ?_OptionsStorage@?1??__local_stdio_scanf_options@@9@4_KA 00000001800222b0     MSVCRT:default_local_stdio_options.obj
 0003:0001b2b8       __favor                    00000001800222b8     MSVCRT:cpu_disp.obj
 0003:0001b2c0       __dyn_tls_init_callback    00000001800222c0     <common>

 entry point at        0001:000020f0

 Static symbols

 0000:fffdb000       .debug$S                   0000000180000000     objmonusage006.exp
 0000:fffdb000       .debug$S                   0000000180000000     vcruntime:VCRUNTIME140.dll
 0000:fffdb000       .debug$S                   0000000180000000     vcruntime:VCRUNTIME140.dll
 0000:fffdb000       .debug$S                   0000000180000000     vcruntime:VCRUNTIME140.dll
 0000:fffdb000       .debug$S                   0000000180000000     vcruntime:VCRUNTIME140.dll
 0000:fffdb000       .debug$S                   0000000180000000     vcruntime:VCRUNTIME140.dll
 0000:fffdb000       .debug$S                   0000000180000000     vcruntime:VCRUNTIME140.dll
 0000:fffdb000       .debug$S                   0000000180000000     vcruntime:VCRUNTIME140.dll
 0000:fffdb000       .debug$S                   0000000180000000     ucrt:api-ms-win-crt-convert-l1-1-0.dll
 0002:ffffc000       .idata$6                   0000000180000000     ucrt:api-ms-win-crt-convert-l1-1-0.dll
 0000:fffdb000       .debug$S                   0000000180000000     ucrt:api-ms-win-crt-heap-l1-1-0.dll
 0000:fffdb000       .debug$S                   0000000180000000     ucrt:api-ms-win-crt-heap-l1-1-0.dll
 0000:fffdb000       .debug$S                   0000000180000000     ucrt:api-ms-win-crt-heap-l1-1-0.dll
 0000:fffdb000       .debug$S                   0000000180000000     ucrt:api-ms-win-crt-heap-l1-1-0.dll
 0002:ffffc000       .idata$6                   0000000180000000     ucrt:api-ms-win-crt-heap-l1-1-0.dll
 0000:fffdb000       .debug$S                   0000000180000000     ucrt:api-ms-win-crt-runtime-l1-1-0.dll
 0000:fffdb000       .debug$S                   0000000180000000     ucrt:api-ms-win-crt-runtime-l1-1-0.dll
 0000:fffdb000       .debug$S                   0000000180000000     ucrt:api-ms-win-crt-runtime-l1-1-0.dll
 0000:fffdb000       .debug$S                   0000000180000000     ucrt:api-ms-win-crt-runtime-l1-1-0.dll
 0000:fffdb000       .debug$S                   0000000180000000     ucrt:api-ms-win-crt-runtime-l1-1-0.dll
 0000:fffdb000       .debug$S                   0000000180000000     ucrt:api-ms-win-crt-runtime-l1-1-0.dll
 0000:fffdb000       .debug$S                   0000000180000000     ucrt:api-ms-win-crt-runtime-l1-1-0.dll
 0000:fffdb000       .debug$S                   0000000180000000     ucrt:api-ms-win-crt-runtime-l1-1-0.dll
 0000:fffdb000       .debug$S                   0000000180000000     ucrt:api-ms-win-crt-runtime-l1-1-0.dll
 0000:fffdb000       .debug$S                   0000000180000000     ucrt:api-ms-win-crt-runtime-l1-1-0.dll
 0000:fffdb000       .debug$S                   0000000180000000     ucrt:api-ms-win-crt-runtime-l1-1-0.dll
 0000:fffdb000       .debug$S                   0000000180000000     ucrt:api-ms-win-crt-runtime-l1-1-0.dll
 0000:fffdb000       .debug$S                   0000000180000000     ucrt:api-ms-win-crt-runtime-l1-1-0.dll
 0000:fffdb000       .debug$S                   0000000180000000     ucrt:api-ms-win-crt-runtime-l1-1-0.dll
 0000:fffdb000       .debug$S                   0000000180000000     ucrt:api-ms-win-crt-runtime-l1-1-0.dll
 0000:fffdb000       .debug$S                   0000000180000000     ucrt:api-ms-win-crt-runtime-l1-1-0.dll
 0000:fffdb000       .debug$S                   0000000180000000     ucrt:api-ms-win-crt-stdio-l1-1-0.dll
 0000:fffdb000       .debug$S                   0000000180000000     ucrt:api-ms-win-crt-stdio-l1-1-0.dll
 0000:fffdb000       .debug$S                   0000000180000000     ucrt:api-ms-win-crt-stdio-l1-1-0.dll
 0000:fffdb000       .debug$S                   0000000180000000     ucrt:api-ms-win-crt-stdio-l1-1-0.dll
 0000:fffdb000       .debug$S                   0000000180000000     ucrt:api-ms-win-crt-stdio-l1-1-0.dll
 0000:fffdb000       .debug$S                   0000000180000000     ucrt:api-ms-win-crt-stdio-l1-1-0.dll
 0000:fffdb000       .debug$S                   0000000180000000     ucrt:api-ms-win-crt-stdio-l1-1-0.dll
 0000:fffdb000       .debug$S                   0000000180000000     ucrt:api-ms-win-crt-stdio-l1-1-0.dll
 0000:fffdb000       .debug$S                   0000000180000000     ucrt:api-ms-win-crt-stdio-l1-1-0.dll
 0000:fffdb000       .debug$S                   0000000180000000     ucrt:api-ms-win-crt-stdio-l1-1-0.dll
 0000:fffdb000       .debug$S                   0000000180000000     ucrt:api-ms-win-crt-string-l1-1-0.dll
 0000:fffdb000       .debug$S                   0000000180000000     ucrt:api-ms-win-crt-string-l1-1-0.dll
 0000:fffdb000       .debug$S                   0000000180000000     ucrt:api-ms-win-crt-string-l1-1-0.dll
 0000:fffdb000       .debug$S                   0000000180000000     ucrt:api-ms-win-crt-string-l1-1-0.dll
 0000:fffdb000       .debug$S                   0000000180000000     ucrt:api-ms-win-crt-string-l1-1-0.dll
 0000:fffdb000       .debug$S                   0000000180000000     ucrt:api-ms-win-crt-string-l1-1-0.dll
 0000:fffdb000       .debug$S                   0000000180000000     ucrt:api-ms-win-crt-string-l1-1-0.dll
 0000:fffdb000       .debug$S                   0000000180000000     ucrt:api-ms-win-crt-string-l1-1-0.dll
 0000:fffdb000       .debug$S                   0000000180000000     kernel32:KERNEL32.dll
 0000:fffdb000       .debug$S                   0000000180000000     kernel32:KERNEL32.dll
 0000:fffdb000       .debug$S                   0000000180000000     kernel32:KERNEL32.dll
 0000:fffdb000       .debug$S                   0000000180000000     kernel32:KERNEL32.dll
 0000:fffdb000       .debug$S                   0000000180000000     kernel32:KERNEL32.dll
 0000:fffdb000       .debug$S                   0000000180000000     kernel32:KERNEL32.dll
 0000:fffdb000       .debug$S                   0000000180000000     kernel32:KERNEL32.dll
 0000:fffdb000       .debug$S                   0000000180000000     kernel32:KERNEL32.dll
 0000:fffdb000       .debug$S                   0000000180000000     kernel32:KERNEL32.dll
 0000:fffdb000       .debug$S                   0000000180000000     kernel32:KERNEL32.dll
 0000:fffdb000       .debug$S                   0000000180000000     kernel32:KERNEL32.dll
 0000:fffdb000       .debug$S                   0000000180000000     kernel32:KERNEL32.dll
 0000:fffdb000       .debug$S                   0000000180000000     kernel32:KERNEL32.dll
 0000:fffdb000       .debug$S                   0000000180000000     kernel32:KERNEL32.dll
 0000:fffdb000       .debug$S                   0000000180000000     kernel32:KERNEL32.dll
 0000:fffdb000       .debug$S                   0000000180000000     kernel32:KERNEL32.dll
 0000:fffdb000       .debug$S                   0000000180000000     kernel32:KERNEL32.dll
 0000:fffdb000       .debug$S                   0000000180000000     kernel32:KERNEL32.dll
 0000:fffdb000       .debug$S                   0000000180000000     kernel32:KERNEL32.dll
 0000:fffdb000       .debug$S                   0000000180000000     kernel32:KERNEL32.dll
 0000:fffdb000       .debug$S                   0000000180000000     kernel32:KERNEL32.dll
 0000:fffdb000       .debug$S                   0000000180000000     kernel32:KERNEL32.dll
 0000:fffdb000       .debug$S                   0000000180000000     kernel32:KERNEL32.dll
 0000:fffdb000       .debug$S                   0000000180000000     kernel32:KERNEL32.dll
 0000:fffdb000       .debug$S                   0000000180000000     kernel32:KERNEL32.dll
 0000:fffdb000       .debug$S                   0000000180000000     kernel32:KERNEL32.dll
 0000:fffdb000       .debug$S                   0000000180000000     kernel32:KERNEL32.dll
 0000:fffdb000       .debug$S                   0000000180000000     kernel32:KERNEL32.dll
 0001:00000d8c       addRefToVerify             0000000180001d8c f   libobjmonusage006.obj
 0001:00000e00       agentThreadWrapper         0000000180001e00 f   libobjmonusage006.obj
 0001:00000fd8       file_basename              0000000180001fd8 f   libobjmonusage006.obj
 0001:00001600       startAgentThreadWrapper    0000000180002600 f   libobjmonusage006.obj
 0001:0000192c       syncDebuggeeStatus         000000018000292c f   libobjmonusage006.obj
 0001:00001bb4       capture_previous_context   0000000180002bb4 f   MSVCRT:gs_report.obj
 0001:00001c28       ?__scrt_initialize_thread_safe_statics@@YAHXZ 0000000180002c28 f   MSVCRT:thread_safe_statics.obj
 0001:00001cf8       ?__scrt_uninitialize_thread_safe_statics@@YAXXZ 0000000180002cf8 f   MSVCRT:thread_safe_statics.obj
 0001:00001da0       $$000000                   0000000180002da0     MSVCRT:amdsecgs.obj
 0001:00001dd0       ?dllmain_crt_dispatch@@YAHQEAUHINSTANCE__@@KQEAX@Z 0000000180002dd0 f   MSVCRT:dll_dllmain.obj
 0001:00001e20       ?dllmain_crt_process_attach@@YAHQEAUHINSTANCE__@@QEAX@Z 0000000180002e20 f   MSVCRT:dll_dllmain.obj
 0001:00001f38       ?dllmain_crt_process_detach@@YAH_N@Z 0000000180002f38 f   MSVCRT:dll_dllmain.obj
 0001:00001fbc       ?dllmain_dispatch@@YAHQEAUHINSTANCE__@@KQEAX@Z 0000000180002fbc f   MSVCRT:dll_dllmain.obj
 0001:000029d0       $$000000                   00000001800039d0     MSVCRT:guard_dispatch.obj
 0001:000029f0       $$000000                   00000001800039f0     MSVCRT:guard_xfg_dispatch.obj
 0001:00002a06       ?fin$0@?0??dllmain_crt_process_attach@@YAHQEAUHINSTANCE__@@QEAX@Z@4HA 0000000180003a06 f   MSVCRT:dll_dllmain.obj
 0001:00002a1d       ?fin$0@?0??dllmain_crt_process_detach@@YAH_N@Z@4HA 0000000180003a1d f   MSVCRT:dll_dllmain.obj
 0001:00002a36       ?fin$1@?0??dllmain_crt_process_detach@@YAH_N@Z@4HA 0000000180003a36 f   MSVCRT:dll_dllmain.obj
 0001:00002a4a       ?filt$0@?0??dllmain_dispatch@@YAHQEAUHINSTANCE__@@KQEAX@Z@4HA 0000000180003a4a f   MSVCRT:dll_dllmain.obj
 0001:00002a80       __scrt_is_nonwritable_in_current_image$filt$0 0000000180003a80 f   MSVCRT:utility.obj
 0002:000001e0       ?__scrt_initialize_tss_var@@3P6AHXZEA 00000001800041e0     MSVCRT:thread_safe_statics.obj
 0002:00000300       ?opcLengths@@3QBEB         0000000180004300     libobjmonusage006.obj
 0002:000019e0       GS_ExceptionPointers       00000001800059e0     MSVCRT:gs_report.obj
 0002:000020a8       $unwind$fprintf            00000001800060a8     libobjmonusage006.obj
 0002:000020b4       $unwind$printf             00000001800060b4     libobjmonusage006.obj
 0002:000020c0       $unwind$?NewObject@JNIEnv_@@QEAAPEAV_jobject@@PEAV_jclass@@PEAU_jmethodID@@ZZ 00000001800060c0     libobjmonusage006.obj
 0002:000020c0       $unwind$nsk_lcomplain      00000001800060c0     libobjmonusage006.obj
 0002:000020c0       $unwind$nsk_ldisplay       00000001800060c0     libobjmonusage006.obj
 0002:000020c8       $unwind$nsk_lvdisplay      00000001800060c8     libobjmonusage006.obj
 0002:000020c8       $unwind$_RTC_Initialize    00000001800060c8     MSVCRT:initsect.obj
 0002:000020c8       $unwind$_RTC_Terminate     00000001800060c8     MSVCRT:initsect.obj
 0002:000020c8       $unwind$?__scrt_initialize_thread_safe_statics@@YAHXZ 00000001800060c8     MSVCRT:thread_safe_statics.obj
 0002:000020d4       $unwind$nsk_lvcomplain     00000001800060d4     libobjmonusage006.obj
 0002:000020ec       $unwind$nsk_ltrace         00000001800060ec     libobjmonusage006.obj
 0002:000020ec       $unwind$__report_gsfailure 00000001800060ec     MSVCRT:gs_report.obj
 0002:000020f4       $unwind$Agent_Initialize   00000001800060f4     libobjmonusage006.obj
 0002:000020f4       $unwind$nsk_lvtrace        00000001800060f4     libobjmonusage006.obj
 0002:000020f4       $unwind$__raise_securityfailure 00000001800060f4     MSVCRT:gs_report.obj
 0002:000020f4       $unwind$__scrt_initialize_crt 00000001800060f4     MSVCRT:utility.obj
 0002:000020f4       $unwind$__scrt_initialize_onexit_tables 00000001800060f4     MSVCRT:utility.obj
 0002:000020f4       $unwind$__scrt_release_startup_lock 00000001800060f4     MSVCRT:utility.obj
 0002:000020f4       $unwind$__scrt_uninitialize_crt 00000001800060f4     MSVCRT:utility.obj
 0002:000020f4       $unwind$_onexit            00000001800060f4     MSVCRT:utility.obj
 0002:000020fc       $unwind$nsk_lverify        00000001800060fc     libobjmonusage006.obj
 0002:0000210c       $unwind$nsk_vprintf        000000018000610c     libobjmonusage006.obj
 0002:0000211c       $unwind$nsk_printf         000000018000611c     libobjmonusage006.obj
 0002:00002124       $unwind$?nsk_jni_lverify@@YAHHPEAUJNIEnv_@@HQEBDH1ZZ 0000000180006124     libobjmonusage006.obj
 0002:00002138       $unwind$?nsk_jni_check_exception@@YAHPEAUJNIEnv_@@QEBDH@Z 0000000180006138     libobjmonusage006.obj
 0002:00002154       $unwind$Java_nsk_jvmti_unit_FollowReferences_FollowRefObjects_resetTags 0000000180006154     libobjmonusage006.obj
 0002:00002154       $unwind$addRefToVerify     0000000180006154     libobjmonusage006.obj
 0002:00002154       $unwind$nsk_jvmti_resetAgentData 0000000180006154     libobjmonusage006.obj
 0002:00002154       $unwind$__scrt_initialize_default_local_stdio_options 0000000180006154     MSVCRT:default_local_stdio_options.obj
 0002:00002154       $unwind$?dllmain_crt_dispatch@@YAHQEAUHINSTANCE__@@KQEAX@Z 0000000180006154     MSVCRT:dll_dllmain.obj
 0002:00002154       $unwind$DllMain            0000000180006154     MSVCRT:dll_dllmain_stub.obj
 0002:00002154       $unwind$__GSHandlerCheck   0000000180006154     MSVCRT:gshandler.obj
 0002:00002154       $unwind$?__scrt_uninitialize_thread_safe_statics@@YAXXZ 0000000180006154     MSVCRT:thread_safe_statics.obj
 0002:00002154       $unwind$__scrt_acquire_startup_lock 0000000180006154     MSVCRT:utility.obj
 0002:00002154       $unwind$__scrt_dllmain_after_initialize_c 0000000180006154     MSVCRT:utility.obj
 0002:00002154       $unwind$__scrt_dllmain_before_initialize_c 0000000180006154     MSVCRT:utility.obj
 0002:00002154       $unwind$__scrt_dllmain_crt_thread_attach 0000000180006154     MSVCRT:utility.obj
 0002:00002154       $unwind$__scrt_dllmain_crt_thread_detach 0000000180006154     MSVCRT:utility.obj
 0002:00002154       $unwind$__scrt_dllmain_uninitialize_c 0000000180006154     MSVCRT:utility.obj
 0002:00002154       $unwind$__scrt_dllmain_uninitialize_critical 0000000180006154     MSVCRT:utility.obj
 0002:00002154       $unwind$atexit             0000000180006154     MSVCRT:utility.obj
 0002:0000215c       $unwind$nsk_jvmti_lverify  000000018000615c     libobjmonusage006.obj
 0002:00002170       $unwind$exitOnError        0000000180006170     libobjmonusage006.obj
 0002:00002180       $unwind$Java_nsk_share_jvmti_ArgumentHandler_getAgentOptionsString 0000000180006180     libobjmonusage006.obj
 0002:00002194       $unwind$Java_nsk_jvmti_unit_FollowReferences_FollowRefObjects_getTag 0000000180006194     libobjmonusage006.obj
 0002:00002194       $unwind$Java_nsk_share_jvmti_DebugeeClass_checkStatus 0000000180006194     libobjmonusage006.obj
 0002:00002194       $unwind$agentThreadWrapper 0000000180006194     libobjmonusage006.obj
 0002:000021a4       $unwind$startAgentThreadWrapper 00000001800061a4     libobjmonusage006.obj
 0002:000021c0       $unwind$syncDebuggeeStatus 00000001800061c0     libobjmonusage006.obj
 0002:000021c0       $unwind$__scrt_dllmain_exception_filter 00000001800061c0     MSVCRT:utility.obj
 0002:000021d4       $unwind$Java_nsk_share_jvmti_DebugeeClass_resetAgentData 00000001800061d4     libobjmonusage006.obj
 0002:000021dc       $unwind$MA_checkStatus     00000001800061dc     libobjmonusage006.obj
 0002:000021f0       $unwind$Java_nsk_jvmti_unit_FollowReferences_FollowRefObjects_setTag 00000001800061f0     libobjmonusage006.obj
 0002:00002208       $unwind$Java_nsk_jvmti_unit_FollowReferences_FollowRefObjects_addRefToVerify 0000000180006208     libobjmonusage006.obj
 0002:00002224       $unwind$Java_nsk_jvmti_GetObjectMonitorUsage_objmonusage006_check 0000000180006224     libobjmonusage006.obj
 0002:0000222c       $unwind$capture_previous_context 000000018000622c     MSVCRT:gs_report.obj
 0002:00002238       $unwind$__GSHandlerCheckCommon 0000000180006238     MSVCRT:gshandler.obj
 0002:00002240       $xdatasym                  0000000180006240     MSVCRT:amdsecgs.obj
 0002:00002244       $unwind$?dllmain_crt_process_attach@@YAHQEAUHINSTANCE__@@QEAX@Z 0000000180006244     MSVCRT:dll_dllmain.obj
 0002:00002280       $unwind$?fin$0@?0??dllmain_crt_process_attach@@YAHQEAUHINSTANCE__@@QEAX@Z@4HA 0000000180006280     MSVCRT:dll_dllmain.obj
 0002:00002280       $unwind$?fin$0@?0??dllmain_crt_process_detach@@YAH_N@Z@4HA 0000000180006280     MSVCRT:dll_dllmain.obj
 0002:00002280       $unwind$?fin$1@?0??dllmain_crt_process_detach@@YAH_N@Z@4HA 0000000180006280     MSVCRT:dll_dllmain.obj
 0002:00002288       $unwind$?dllmain_crt_process_detach@@YAH_N@Z 0000000180006288     MSVCRT:dll_dllmain.obj
 0002:000022dc       $unwind$?dllmain_dispatch@@YAHQEAUHINSTANCE__@@KQEAX@Z 00000001800062dc     MSVCRT:dll_dllmain.obj
 0002:00002304       $unwind$?filt$0@?0??dllmain_dispatch@@YAHQEAUHINSTANCE__@@KQEAX@Z@4HA 0000000180006304     MSVCRT:dll_dllmain.obj
 0002:0000230c       $unwind$_DllMainCRTStartup 000000018000630c     MSVCRT:dll_dllmain.obj
 0002:0000231c       $unwind$__scrt_is_nonwritable_in_current_image 000000018000631c     MSVCRT:utility.obj
 0002:0000233c       $unwind$__scrt_is_nonwritable_in_current_image$filt$0 000000018000633c     MSVCRT:utility.obj
 0002:00002344       $unwind$__scrt_fastfail    0000000180006344     MSVCRT:utility_desktop.obj
 0002:00002354       $unwind$__security_init_cookie 0000000180006354     MSVCRT:gs_support.obj
 0002:00002360       $unwind$__isa_available_init 0000000180006360     MSVCRT:cpu_disp.obj
 0002:00002370       $xdatasym                  0000000180006370     MSVCRT:guard_dispatch.obj
 0002:00002378       $xdatasym                  0000000180006378     MSVCRT:guard_xfg_dispatch.obj
 0002:00002380       .edata                     0000000180006380     objmonusage006.exp
 0002:000023a8       rgpv                       00000001800063a8     objmonusage006.exp
 0002:000023e8       rgszName                   00000001800063e8     objmonusage006.exp
 0002:00002428       rgwOrd                     0000000180006428     objmonusage006.exp
 0002:00002448       szName                     0000000180006448     objmonusage006.exp
 0002:0000245b       $N00001                    000000018000645b     objmonusage006.exp
 0002:0000246a       $N00002                    000000018000646a     objmonusage006.exp
 0002:00002477       $N00003                    0000000180006477     objmonusage006.exp
 0002:000024b1       $N00004                    00000001800064b1     objmonusage006.exp
 0002:000024ec       $N00005                    00000001800064ec     objmonusage006.exp
 0002:00002531       $N00006                    0000000180006531     objmonusage006.exp
 0002:0000256e       $N00007                    000000018000656e     objmonusage006.exp
 0002:000025b6       $N00008                    00000001800065b6     objmonusage006.exp
 0002:000025f6       $N00009                    00000001800065f6     objmonusage006.exp
 0002:00002633       $N00010                    0000000180006633     objmonusage006.exp
 0002:0000266e       $N00011                    000000018000666e     objmonusage006.exp
 0002:0000269c       $N00012                    000000018000669c     objmonusage006.exp
 0002:000026cd       $N00013                    00000001800066cd     objmonusage006.exp
 0002:000026fc       $N00014                    00000001800066fc     objmonusage006.exp
 0002:0000272b       $N00015                    000000018000672b     objmonusage006.exp
 0002:00002760       $N00016                    0000000180006760     objmonusage006.exp
 0002:00002b62       .idata$6                   0000000180006b62     kernel32:KERNEL32.dll
 0002:00002bc6       .idata$6                   0000000180006bc6     vcruntime:VCRUNTIME140.dll
 0002:00002d28       .idata$6                   0000000180006d28     ucrt:api-ms-win-crt-runtime-l1-1-0.dll
 0002:00002d4a       .idata$6                   0000000180006d4a     ucrt:api-ms-win-crt-stdio-l1-1-0.dll
 0002:00002d6a       .idata$6                   0000000180006d6a     ucrt:api-ms-win-crt-string-l1-1-0.dll
 0003:00000000       ?codeAttributeName@@3PEBDEB 0000000180007000     libobjmonusage006.obj
 0003:00000008       ?lineNumberAttributeName@@3PEBDEB 0000000180007008     libobjmonusage006.obj
 0003:00000010       ?localVarAttributeName@@3PEBDEB 0000000180007010     libobjmonusage006.obj
 0003:00000018       ?localVarTypeAttributeName@@3PEBDEB 0000000180007018     libobjmonusage006.obj
 0003:00000020       ?stackMapAttributeName@@3PEBDEB 0000000180007020     libobjmonusage006.obj
 0003:00000028       ?callBytes@@3PAEA          0000000180007028     libobjmonusage006.obj
 0003:0000002c       ?allocBytes@@3PAEA         000000018000702c     libobjmonusage006.obj
 0003:0001aad4       redefineAttempted          0000000180021ad4     libobjmonusage006.obj
 0003:0001aad8       nsk_context                0000000180021ad8     libobjmonusage006.obj
 0003:0001aae4       redefineSucceed            0000000180021ae4     libobjmonusage006.obj
 0003:0001aae8       agentFailed                0000000180021ae8     libobjmonusage006.obj
 0003:0001aaec       currentAgentStatus         0000000180021aec     libobjmonusage006.obj
 0003:0001aaf0       context                    0000000180021af0     libobjmonusage006.obj
 0003:0001aba8       agentThread                0000000180021ba8     libobjmonusage006.obj
 0003:0001abb0       agentThreadProc            0000000180021bb0     libobjmonusage006.obj
 0003:0001abb8       agentThreadArg             0000000180021bb8     libobjmonusage006.obj
 0003:0001abc0       agent_data                 0000000180021bc0     libobjmonusage006.obj
 0003:0001abd0       jvmti_env                  0000000180021bd0     libobjmonusage006.obj
 0003:0001abd8       jvm                        0000000180021bd8     libobjmonusage006.obj
 0003:0001abe0       jni_env                    0000000180021be0     libobjmonusage006.obj
 0003:0001abe8       checkStatus_func           0000000180021be8     libobjmonusage006.obj
 0003:0001abf0       ?codeAttributeIndex@@3GA   0000000180021bf0     libobjmonusage006.obj
 0003:0001abf4       ?lineNumberAttributeIndex@@3GA 0000000180021bf4     libobjmonusage006.obj
 0003:0001abf8       ?localVarAttributeIndex@@3GA 0000000180021bf8     libobjmonusage006.obj
 0003:0001abfc       ?localVarTypeAttributeIndex@@3GA 0000000180021bfc     libobjmonusage006.obj
 0003:0001ac00       ?stackMapAttributeIndex@@3GA 0000000180021c00     libobjmonusage006.obj
 0003:0001ac04       ?stackFrameOffset@@3GA     0000000180021c04     libobjmonusage006.obj
 0003:0001ac08       ?mode@@3HA                 0000000180021c08     libobjmonusage006.obj
 0003:0001ac0c       ?constantPoolSize@@3GA     0000000180021c0c     libobjmonusage006.obj
 0003:0001ac10       ?orig@@3PEBEEB             0000000180021c10     libobjmonusage006.obj
 0003:0001ac18       ?gen@@3PEAEEA              0000000180021c18     libobjmonusage006.obj
 0003:0001ac20       ?inputPos@@3PEAEEA         0000000180021c20     libobjmonusage006.obj
 0003:0001ac28       ?endPos@@3PEBEEB           0000000180021c28     libobjmonusage006.obj
 0003:0001ac30       ?genPos@@3PEAEEA           0000000180021c30     libobjmonusage006.obj
 0003:0001ac38       ?markPos@@3PEAEEA          0000000180021c38     libobjmonusage006.obj
 0003:0001ac40       ?constantPool@@3PEAPEADEA  0000000180021c40     libobjmonusage006.obj
 0003:0001ac48       ?constantPoolCount@@3GA    0000000180021c48     libobjmonusage006.obj
 0003:0001ac4c       ?zeroBytes@@3PAEA          0000000180021c4c     libobjmonusage006.obj
 0003:0001ac50       ?codeLength@@3IA           0000000180021c50     libobjmonusage006.obj
 0003:0001ac54       result                     0000000180021c54     libobjmonusage006.obj
 0003:0001ac58       ?map@@3PEAIEA              0000000180021c58     libobjmonusage006.obj
 0003:0001ac60       ?widening@@3PEACEA         0000000180021c60     libobjmonusage006.obj
 0003:0001ac68       jvmti                      0000000180021c68     libobjmonusage006.obj
 0003:0001ac70       caps                       0000000180021c70     libobjmonusage006.obj
 0003:0001ac90       GS_ExceptionRecord         0000000180021c90     MSVCRT:gs_report.obj
 0003:0001ad30       GS_ContextRecord           0000000180021d30     MSVCRT:gs_report.obj
 0003:0001b200       ?g_tss_cv@@3U_RTL_CONDITION_VARIABLE@@A 0000000180022200     MSVCRT:thread_safe_statics.obj
 0003:0001b208       ?g_tss_event@@3PEAXEA      0000000180022208     MSVCRT:thread_safe_statics.obj
 0003:0001b210       ?g_tss_mutex@@3U_RTL_CRITICAL_SECTION@@A 0000000180022210     MSVCRT:thread_safe_statics.obj
 0003:0001b238       ?g_sleep_condition_variable_cs@@3P6AHPEAU_RTL_CONDITION_VARIABLE@@PEAU_RTL_CRITICAL_SECTION@@K@ZEA 0000000180022238     MSVCRT:thread_safe_statics.obj
 0003:0001b240       ?g_wake_all_condition_variable@@3P6AXPEAU_RTL_CONDITION_VARIABLE@@@ZEA 0000000180022240     MSVCRT:thread_safe_statics.obj
 0003:0001b24c       ?__proc_attached@@3HA      000000018002224c     MSVCRT:dll_dllmain.obj
 0003:0001b260       ?is_initialized_as_dll@@3_NA 0000000180022260     MSVCRT:utility.obj
 0003:0001b261       ?module_local_atexit_table_initialized@@3_NA 0000000180022261     MSVCRT:utility.obj
 0003:0001b268       ?module_local_atexit_table@@3U_onexit_table_t@@A 0000000180022268     MSVCRT:utility.obj
 0003:0001b280       ?module_local_at_quick_exit_table@@3U_onexit_table_t@@A 0000000180022280     MSVCRT:utility.obj
